:020000020000FC
:100000000C9434000C946B0D0C946B0D0C946B0DD4
:100010000C946B0D0C946B0D0C946B0D0C94020CEA
:100020000C946B0D0C946B0D0C946B0D0C946B0D70
:100030000C946B0D0C946B0D0C946B0D0C946B0D60
:100040000C946B0D0C946B0D0C946B0D0C946B0D50
:100050000C946B0D0C946B0D0C946B0D0C946B0D40
:100060000C946B0D0C946B0DA8950FEF0DBF04E075
:100070000EBF0E94C90C0E94600278940E94180171
:100080000FEFC02E0E94DD000E947C010C943D0009
:100090000590002009F0089500E00093BD040C9441
:1000A000C007E8EDFAE10E944800071671F40E94CB
:1000B0004800061659F40E944800051641F431968E
:1000C0000591F491E02F0995089531963196309677
:1000D0000C94530070EF60EF41E018810E94A10082
:1000E000013021F40E9495000C946A00512F0E9467
:1000F00095001D30A9F03D2C18811D3089F00E941B
:10010000A1003D1441F4762F652F512F0E949500D8
:100110004395433089F718810E94A1003D1409F0EE
:1001200008950E9495000C948B00DB1541F4CA15CC
:1001300031F404E00093BD040C94C00708952197A6
:1001400008951F9300271D3011F40C94C4001F75EF
:10015000103011F40C94AE001C3019F401E00C9432
:10016000C500103112F40C94C5001B3512F00C942C
:10017000C50010341AF003E00C94C5001A3112F4D3
:1001800022F402E00C94C50004E0D02E1F910895E3
:10019000CF3329F447E00E9406010C94E20048E0C6
:1001A0000E941F0140E20E941F01412F0E941F0177
:1001B000C3951DE018830C94E2004EE30E940601F3
:1001C000D4E0CFE30E942601183011F31F3701F36A
:1001D0001A3011F40C94E20018831D3069F0C0301D
:1001E00029F447E00E9406010C94E200CA95412FD1
:1001F0000E941F010C94E20008950E9428028F9330
:10020000492F0E9406014F9101D008950090C0002F
:1002100005FE0C9406010E94E705B6FF0C9415013B
:100220000090C00007FEFCCFBF7B4093C60008953E
:100230004DE00E9406014AE00E94060108954D30FB
:1002400019F40E94180108950C9406018895000085
:100250000091C00007FF0C9426011091C60008957C
:100260000E9435010E94180108954591442321F10F
:10027000483F21F40E945D010C943501493F31F45F
:10028000159045910E9477010C9435014A3F21F465
:100290000E9418010C9435014B3F51F4EF93FF93EA
:1002A000EEE2F0E20E943501FF91EF910C943501EE
:1002B0000E9406010C9435010895EF93FF931124D9
:1002C00045914A3049F04C3039F04A3F29F0493FD6
:1002D00019F013940C9460011A944CE3141A1194BD
:1002E000169440E20E947701FF91EF9108950E94D9
:1002F00006011A94E1F70895D4E0CFE30FEFA02EA2
:1003000004E0B02E18810E94A100023011F40C9478
:1003100064060E941801A1600C948F01AE7F8DB716
:100320008F3C28F408E00093BD040C94C0070E94A1
:100330006A005D30F9F05B33E9F0032D023049F4D7
:100340007F706F705F700E9443020E94D0010C9416
:100350008F017F756F755F75413039F4032D033060
:1003600021F40E94BC010C948F010E9451005D3069
:1003700009F00895A160089551545A312AF005E01A
:100380000093BD040C94C007505CA0FF19F40E94B8
:10039000D0010895F4E0E52F50810E94D001089526
:1003A0000F93F3E0EC2D5083CA940C2D033F28F4F7
:1003B00006E00093BD040C94C0070F9108950F93BD
:1003C000C3940C2D00302AF007E00093BD040C9478
:1003D000C007F3E0EC2D50810F9108950E94DF01DA
:1003E00007E005175AF001E0503021F0000F5A9550
:1003F0000C94F401502F0E94D00108950AE000935C
:10040000BD040E94C007703049F0705D472F0E9404
:100410000601603019F440E30E940601603021F0CB
:10042000605D462F0E940601505D452F0E94060127
:10043000089577276627545618F073950C941B027D
:100440005C595A5018F063950C942102565F089538
:10045000982F9695969596959695905D9A3308F077
:10046000995F8F70805D8A3308F0895F089596FDEB
:10047000975F9F7086FD875F8F70990F990F990F17
:10048000990F892B08957330B2F4723032F06630D0
:1004900092F4653012F0563072F4662321F00AE0CF
:1004A000500F6A9581F7772309F4089504E688943C
:1004B000500F7A95C0F701E00093BD040C94C0077B
:1004C000E6E7FDE10E94300108950E941801F3E083
:1004D000E4EFC091B904D091BA04FD1711F4EC1700
:1004E00031F040810E941F0131970C946D020E94EF
:1004F00018010E941801EAEFFFE10E9435015091B6
:10050000B9047091BA04505071400E94D001572F25
:100510000E9419020E940302E8E0F0E20E94350105
:100520000E94DF010E9419020E9403020E9418012A
:100530000895AE7F0E948F010E94DF010E94190280
:100540000E9403020E94180108950E948E0144E255
:100550000E9406010E94DF01852F0E94FD000E947B
:1005600018010895AE7F0E948F010E94DF01052FC0
:100570000E94DF01F4E0E52F00830895A2FF0C94B0
:100580007003AE7F0E948F010E94DF01452E0E9402
:10059000DF01652F0E94DF01552EF4E0E52F608317
:1005A000A062A860AA7F0895F4E0E52D00810415FB
:1005B00019F003950083A06108950E948E010E94A6
:1005C000DF01052F0E94DF01501721F055270E94FF
:1005D000D00108955FEF0E94D00108950E948E011E
:1005E00050E000B605FE51E00E94D00108950E943F
:1005F0008E010EEF0C1949F00E94DF015F930E94FB
:10060000DF01F52FEF910C9409030E94DF01E52F24
:10061000FF2750810E94D00108950E948E010DEFA6
:100620000C1961F00E94DF015F930E94DF015F936C
:100630000E94DF01FF91EF910C9425030E94DF01DE
:10064000052F0E94DF01E02FFF27508308950E94AD
:100650008E010E94DF01052F0E94DF01509F1120B3
:10066000F09921F4502D0E94D00108950FE00093DD
:10067000BD040E94C0070E948E010E94DF01552325
:10068000F099B9F0052F0E94DF01652F771B59E023
:10069000661F5A9551F0771F701B20F4700F8894D5
:1006A0000C94480308940C944803562F0E94D001E0
:1006B000089501E10093BD040E94C0070E948E01CD
:1006C0000E94DF01052F0E94DF01500FF09918F002
:1006D0000E94D00108950FE00093BD040E94C0075E
:1006E0000E948E010E94DF01052F0E94DF01501B36
:1006F000F0991BF00E94D001089500E10093BD0421
:100700000E94C0070E948E010E94DF01052F0E94F7
:10071000DF0150230E94D00108950E948E010E94A3
:10072000DF0156950E94D00108950E948E010E941B
:10073000DF01550F0E94D00108950E948E010E9492
:10074000DF01052F0E94DF01502B0E94D001089588
:100750000E948E010E94DF01052F0E94DF015027B9
:100760000E94D00108950E948E010E94DF015095E1
:100770000E94D00108950E948E010E94DF015195D0
:100780000E94D001089551E00E94D00108950E9476
:100790008E010E94DF01052F0E94DF0150170C948B
:1007A000D9030E948E010E94DF01052F0E94DF0104
:1007B000051750E042F739F30E94D00108950E94D6
:1007C0008E010E94DF01552309F0A26008950DB744
:1007D0000E5F0DBF0895A46008950E948E010895D4
:1007E000B260089598810E94950088810E94370226
:1007F000582F0E94D0010E9495000E948E010895FA
:100800000E948E010E94DF01CF93DF93D0E5C9EFF4
:10081000CA950000E9F7DA950000C9F75A95B1F7D3
:10082000DF91CF91089555270E94D0010E948E013B
:100830000E94DF0101E005172AF0F09850FF0895AB
:10084000F09A08950CE00093BD040E94C0070E9436
:100850008E010E94DF01452FF3E0E4EF8091B9049F
:100860009091BA040C943F04F91711F48E1708F50F
:1008700000810D3019F031970C94340431975527CD
:1008800066277727F91711F48E1798F410810E94C4
:10089000A100023031F4762F652F512F31970C943F
:1008A00042047F706F705F700E9443024517E1F64B
:1008B000089509E00093BD040C94C0070E9427042A
:1008C000DF2FCE2F08950E942704A06C0895B2FF59
:1008D0000C946C04B1600895B26008950E948E017A
:1008E0000E94DF01452F0E940601089588950000AF
:1008F0000091C00007FFFACF5091C600533009F4B1
:10090000B2600E94D00108950E948E010E94DF0112
:1009100008E040E3551F08F441E378DC0A95C9F785
:100920000E941801089504EB5091BE04579508F4F5
:1009300050275093BE040E94D0010895D3E0C4EF25
:100940000FEFC02EA1600E94E705A5FF0C94AB0439
:100950006C2E7D2EAF7DA4FF0C94B104D72DC62D37
:10096000AF7EA6FF0C94B904D093BC04C093BB0423
:10097000AF7BA7FF0C94C004DF2FCE2FB460AF77FE
:10098000B0FF0C94C804C091BB04D091BC04BA7FE2
:10099000B1FF0C94D2040E94E205C091B904D09139
:1009A000BA04BD7F0091BA04D01721F40091B904B4
:1009B0000C17A0F418810E94A100A1FF0C94E5047B
:1009C000043019F021970C94A004AD7F023019F483
:1009D00021970C94A0040E948F01B2CF0895F3E0F8
:1009E000E4EFF093BA04E093B9040FEFC02EAA2706
:1009F000BB27F1E0E0E000E00193F330E8F3E43FEF
:100A0000D9F7F4E0E0E400E00193F430E8F3EA35EC
:100A1000D9F70E941801EEE2FDE10E94300108952D
:100A2000EAE3FFE10E943501E4E6FFE10E943501BF
:100A300000E1202EF3E0E4EF8F2F0E94FD008E2FC7
:100A40000E94FD004AE30E94060140E20E94060166
:100A5000F13011F4E030D9F080810E94FD0040E2D5
:100A60000E94060131972A9481F40E9418018F2F69
:100A70000E94FD008E2F0E94FD004AE30E940601A5
:100A800040E20E94060100E1202E0C9428050E94FD
:100A900018010E941801E0E8FFE10E9435018091F1
:100AA000BA040E94FD008091B9040E94FD000E94DA
:100AB0001801EAE3FFE10E9435010E941801089540
:100AC000EAE3FFE10E943501E4E5FFE10E94350120
:100AD00000E1202EF1E0EFEF8F2F0E94FD008E2F1E
:100AE0000E94FD004AE30E94060140E20E940601C6
:100AF0000F93E03000E0F0070F91F1F0F2BDE1BD9F
:100B0000F89A80B50E94FD0040E20E9406013197EC
:100B10002A9481F40E9418018F2F0E94FD008E2FCD
:100B20000E94FD004AE30E94060140E20E94060185
:100B300000E1202E0C9478050E941801EAE3FFE101
:100B40000E9435010E9418010895EAE3FFE10E9426
:100B50003501E0E4FFE10E94350100E1202EE0E4F0
:100B6000F4E08F2F0E94FD008E2F0E94FD004AE3CB
:100B70000E94060140E20E940601EA35D1F081910F
:100B80000E94FD0040E20E9406012A9481F40E9426
:100B900018018F2F0E94FD008E2F0E94FD004AE356
:100BA0000E94060140E20E94060100E1202E0C9402
:100BB000BD050E941801EAE3FFE10E9435010E9491
:100BC00018010895E2EFFFE10E94350108950090B9
:100BD000C00007FE0C94F7050091C600033111F424
:100BE000B06408950091C600033009F4B26008951E
:100BF000DF93D2E0DA950000E9F7DF910895DF9303
:100C0000D4E1DA950000E9F7DF910895CF93DF93FF
:100C1000D0E5C3EFCA950000000000000000D1F746
:100C2000CFEFCA95000000000000D9F7CCEFCA95BD
:100C30000000000000000000D1F716F06894E9CF32
:100C4000DA95E89431F7DF91CF910895D4E0CFE3BE
:100C5000552788279927BF7D1881CA9583951D3010
:100C600051F00E94A100023041F0B0620130A1F3C6
:100C700093950C942C06092F0895B5FF53950C9469
:100C80002C0604E00093BD040C94C00702E000931E
:100C9000BD040C94C0070BE00093BD0471C17F70CC
:100CA0006F705F700E9443020895D4E0CFE3E0309C
:100CB00069F308810083319721970D30C1F7F093D4
:100CC000BA04E093B90408950E942606543018F738
:100CD0008091B9049091BA04933021F4843F11F4C7
:100CE0000C94D306D4E0CFE3552766277727CA159F
:100CF00042F218810E94A100023031F4762F652F54
:100D0000512F21970C9477060E944F06452EE091B3
:100D1000B904F091BA04B77FBF7E772766275527BD
:100D200055243196F33011F4E53F69F010810E94AB
:100D3000A100043041F0023081F75394562F672F01
:100D4000712F0C949106052D033031F05394562FDA
:100D5000672F70E00C94A306B4FD0C94B206B0614A
:100D60000C948D060E944F064516F1F118F4B860F8
:100D70007F2E6E2EF33029F4E53F19F4B3FF0C9467
:100D8000D306B3FF0C94C806541538F40C941E0710
:100D9000F33019F6E53F09F60895F33021F4E53F05
:100DA00011F40C941E070E942606003009F40895E1
:100DB000D4E0CFE3E091B904F091BA04F13021F42A
:100DC000E03011F40C94EF060881008331972197ED
:100DD0000D30A1F7F093BA04E093B904089502E04E
:100DE0000093BD040C94C0073197EF01D13021F47A
:100DF000C03011F40C944106088121970D30B1F7F1
:100E00000E2F0C1B8091B9049091BA04800F80932F
:100E1000B90418F493959093B904D13011F4C0300B
:100E200031F008810083219731970C940D070E94BF
:100E30002606003011F00C94640608950E942606E0
:100E4000003071F10091BA04013029F40091B90425
:100E50000050081720F2E091B904F091BA04DF2F96
:100E6000CE2FC81BD040D093BA04C093B904F71555
:100E700021F4E61511F40C944307008108832196B0
:100E800031960C943707D4E0CFE3F72DE62D319758
:100E9000088100830D3021F0319721970C94480789
:100EA0000895D3E0CFEFE091B904F091BA04CE1BDE
:100EB000DF0BF1E0EFEFEC17FD072CF4ECE9FFE1BD
:100EC0000E9430010895ECEBFFE10E9430010FEF2A
:100ED000C02E5091B9040E94D0015091BA040E94D2
:100EE000D001D3E0CFEFF1E0EFEF0881F9990C9456
:100EF0007607F2BDE1BD00BDFA9AF99AD13011F43E
:100F0000C03051F031970F93E03000E0F0070F91BF
:100F100019F021970C9475070895EEEDFFE10E94FA
:100F200030010E94EF04D3E0CFEFEFEFF1E0F99949
:100F30000C949707F2BDE1BDF89A00B50883D13053
:100F400011F4C03021F0319721970C9497070DEFE1
:100F5000C02E0E94DF015093BA04F52F0E94DF01DA
:100F60005093B904E52F0F93EF3F03E0F0070F9183
:100F700031F4EEECFFE10E9430010E94EF0408958D
:100F80000E9418010091BD04000FE4EBFFE0E00FA8
:100F90000591F491E02FEE1FFF1F0E9435010FEF26
:100FA0000DBF04E00EBF0FEFC02EA0E0B0E00E9426
:100FB000180163C81B102C104810571075108B10A7
:100FC000A210C110EB1015112F1148115F117811EB
:100FD0009111A411B111BF11CA11D811E811F91161
:100FE000009164000F770093640055270E94D001A0
:100FF0000E948E010E94DF0101E00517A2F002E0CD
:1010000050FD00E20093B800459A449A00270093EF
:10101000B90000950093BB0004E00093BC0004E914
:101020000093BC0008950CE00093BD040E94C0072B
:101030000091BC0002FF0C9447080E948E010E94A0
:10104000DF015093BB0005E80093BC000091BC0099
:1010500007FFFCCF0091B900087F083111F0003480
:1010600041F45091B9005695569556950E94D0017D
:101070000895003239F0083429F002E10093BD04EC
:101080000E94C00704E10093BD040E94C00703E171
:101090000093BD040E94C0070091BC0002FF0C94A5
:1010A00077080E948E010E94DF015093BB0005E883
:1010B0000093BC000091BC0007FFFCCF0091B90079
:1010C000087F083241F45091B900569556955695CF
:1010D0000E94D0010895003329F002E10093BD047D
:1010E0000E94C00704E10093BD040E94C00703E111
:1010F0000093BD040E94C0070091BC0002FF0C9445
:10110000AA0851E00E94D0010E948E010E94DF01D6
:1011100001E0051722F104EC50FF04E80093BC0045
:101120000091BC0007FFFCCF0091B900087F00359B
:1011300029F45091BB000E94D0010895003529F098
:1011400002E10093BD040E94C00704E10093BD04C6
:101150000E94C00703E10093BD040E94C0070CE099
:101160000093BD040E94C0070091BC0002FF0C94D4
:10117000CB0804EA0093BC000091BC0007FFFCCF41
:101180000091B900087F083009F4089502E1009346
:10119000BD040E94C00703E10093BD040E94C00784
:1011A0000091BC0002FF0C94E10804E90093BC002C
:1011B0000FEF0093BB00089502E10093BD040E946D
:1011C000C00703E10093BD040E94C0070091BC006A
:1011D00002FF0C94FF080091BC0004FF0C94F3087C
:1011E00050E80C94FC080091BC0007FFFCCF509124
:1011F000B9005695569556950E94D001089503E181
:101200000093BD040E94C007009164000B7F00930F
:10121000640052E00E94D0010E948E010E94DF0112
:1012200003E005174AF0550F550F0E947A090CB5D7
:10123000037F052B0CBD08950DE00093BD040E94B3
:10124000C0070E948E010E94DF0101E0051752F0E5
:101250000CB500620CBD50FD0C9431090CB50F7D2E
:101260000CBD08950CE00093BD040E94C0070E94CD
:101270008E010E94DF0107E0051782F0052E5370F2
:101280000CB5087F052B0CBD0DB501600DBD02FC32
:101290000C944D090DB50E7F0DBD08950AE0009325
:1012A000BD040E94C0070E948E010E94DF012A989F
:1012B000000000005EBD0DB407FE0C945B095EB536
:1012C00008952A98000000005EBD0DB407FE0C943E
:1012D00065095EB50E94D001089551E00E94D001D9
:1012E0000E948E010E94DF012A9A50FD0C94790918
:1012F0002A98089504B10C6204B905B1046005B9D7
:1013000001E50CBD0DB50E7F0DBD08950091640083
:101310000E7F0093640000E000937B0055270E943D
:10132000D0010E948E010E94DF0100917C00007FAD
:101330005F70052B00937C0006EC00937A0000910F
:101340007A0006FD0C949F0906EC00937A00009148
:101350007A0006FD0C94A709509179000E94D001F3
:10136000089555270E94D0010E948E010E94DF013E
:1013700001E005175AF000917C000F73006250FDE8
:101380000C94C309006C00937C0008950CE000935A
:10139000BD040E94C0070E944F0AEF5DFF4F5081BD
:1013A0000E94D00108950E944F0AEF93FF930E947C
:1013B0008E010E94DF01FF91EF91EF5DFF4F50839F
:1013C00008950E944F0AEF93FF930E948E010E949E
:1013D000EE010E94DF01FF91EF91EF5DFF4F0C9452
:1013E000540A0E944F0AEF93FF930E948E010E94BD
:1013F000EE010E94DF01FF91EF91EF5DFF4F0C9432
:10140000580A0E944F0AEF93FF930E948E010E9498
:10141000DF01FF91EF91EE5DFF4F508308950E9431
:101420004F0AE05EFF4F50810E94D00108950E9454
:101430004F0AEF93FF930E948E010E94EE010E94DB
:10144000DF01FF91EF91EE5DFF4F0C94540A0E9473
:101450004F0AEF93FF930E948E010E94EE010E94BB
:10146000DF01FF91EF91EE5DFF4F0C94580A0E944F
:101470004F0AEF93FF930E948E010E94EE010E949B
:10148000DF01FF91EF91E05EFF4F0081052350E007
:1014900000230FB601FC51E00E94D001089503E043
:1014A0005154509FF00108950081052B0083089549
:1014B000509500810523008308950E948E0101E864
:1014C0000093800009E000938100002700938200D0
:1014D000219A0E94DF010027009389005093880021
:1014E00008950E948E0103E80093800009E00093B4
:1014F0008100002700938200219A0E94DF01052FBE
:101500000E94DF015093890000938800089500270E
:1015100000938000089555270E94D0010E948E01FB
:101520000E94DF0107E005178AF00091BF04087FE1
:10153000502B5093BF04002700936F0006BB00930D
:101540008200009380000093810008950AE00093D8
:10155000BD0416DD51E00E94D0010E948E010E9460
:10156000DF0101E005174AF00091BF040F7750FF3B
:1015700001C000680093BF0408950CE00093BD040F
:10158000FFDCCF93DF936627552756BB609385001A
:1015900050938400B09A0091BF04702F7078C89463
:1015A000771F771F76600770E8EDFAE0E00F099487
:1015B0007AC006C005C004C02AC029C028C04FC0D8
:1015C000033008F005E0709381006093850050932C
:1015D0008400D8E0C3EFCA950000000000000000BE
:1015E000D1F7CFEFCA95000000000000D9F7CCEF8B
:1015F000CA950000000000000000D1F716F06894C2
:10160000E9CFDA95E89431F70A9519F74CC0035001
:10161000033008F005E070938100609385005093DB
:101620008400D0E5C3EFCA95000000000000000070
:10163000D1F7CFEFCA95000000000000D9F7CCEF3A
:10164000CA950000000000000000D1F716F0689471
:10165000E9CFDA95E89431F70A9519F724C0709329
:10166000810060938500509384000AE0D0E5C3EFC9
:10167000CA950000000000000000D1F7CFEFCA9526
:10168000000000000000D9F7CCEFCA950000000070
:1016900000000000D1F716F06894E9CFDA95E894DD
:1016A00031F70A9519F75091840060918500002761
:1016B00000938100B09908C0C9E5D4E068830E9416
:1016C000D001DF91CF910895DF91CF910EE000938B
:1016D000BD0456DC0E948E010E94DF01152F889404
:1016E0000E94820B08950E948E010E94DF01152F37
:1016F00008940E94820B08950E94AC0B512F0E9407
:10170000D001089504B1077E04B905B1086105B997
:1017100079E01C9B0C94890B2D9A259810F02D983C
:10172000259A2C98249A0E94CD0B24982C9A0E94DA
:10173000CD0B1C990C94910B20F02D9A25980C94AC
:10174000A30B2D98259A1C9B0C94A30B25982D9ADE
:10175000111F7A95F1F6089504B1077E04B905B119
:10176000086105B979E01C990C94B30B88941D9B12
:101770000C94C20B08942C98249A1D990C94BD0BC0
:101780000C94C70B2C98249A1D9B0C94C40B249882
:101790002C9A111F7A9539F7089580E590E59A956E
:1017A000F1F78A95D9F70895CF93DF9355270E94D3
:1017B000D0010E948E010E94DF010517F2F050FD5A
:1017C0000C94EE0B0E94B10CC3ECD4E00993099386
:1017D00008835C9A5498DF91CF910895C7E5D4E0CF
:1017E0000E942E0C00270093C604549A5C980E9415
:1017F000910CDF91CF91789408950CE00093BD0493
:101800000E94C0077F937FB77F936F935F93EF939F
:10181000FF93FDE3E091C6045091C3046091C404BA
:101820007091C504E50EF61EE71F5491E093C604BF
:1018300050FF0C94250C00005C9AFF91EF915F9192
:101840006F917F917FBF7F9118955C98FF91EF9189
:101850005F916F917F917FBF7F911895C7E5D4E02D
:1018600077276627552700EF102E08800120029465
:10187000002049F080E0581F90E0691F00E0701FD1
:101880000A940C94380C099012940120002049F01D
:1018900089E9581F99E9691F09E1701F0A940C949E
:1018A000460C0880129401200294002049F08CE537
:1018B000581F9FE8691F02E0701F0A940C94550C92
:1018C000099012940120002049F089E8581F91E402
:1018D000691F00E0701F0A940C94630C0880129436
:1018E00001200294002049F08DE8581F96E0691FFE
:1018F00000E0701F0A940C94720C0880129401206E
:10190000002041F087EA581F90E0691F00E0701F37
:101910000A94B1F75093C3046093C4047093C50450
:101920000895009164000F7B00936400002707BBBB
:101930000093B2000093B0000093B1000093B30095
:101940000093B4000FE40093B30002E00093B000F2
:1019500001E00093B10000917000026000937000FC
:101960000895F894002707BB0093B0000093B100DE
:101970000093B2000093B4000093B3000091700094
:101980000D7F009370000091640000640093640078
:101990000895A89504B7007004BF00916000086125
:1019A0000093600000700093600006E204B900E05C
:1019B00005B900E007B900E008B902E20AB900E0A1
:1019C0000BB900270093BF040EBBF09A54EB0091B3
:1019D000000105270093BE0400E00093C50009E163
:1019E0000093C40008E90093C10001E003BF439ADB
:1019F0000E94FF0533990EC043980E948D070E94F4
:101A00009E040E9418010E941801EEE2FDE10E946E
:101A1000300108950E94EF040895E2E0F0E009E04B
:101A200007BF049106950370003019F4E0E0FCE173
:101A300014C0013019F4E0E0FEE10FC0023019F4E7
:101A4000E0E0FFE10AC0033019F4E0E8FFE105C07F
:101A50000BE00093BD040C94C007EF93FF9308E0E4
:101A6000102EEE1FFF1F05910F3F19F0003009F0F7
:101A700007C01A94C1F705E10093BD040C94C00798
:101A8000E2E1F0E20E943501FF91EF918F2F0E9479
:101A9000FD008E2F0E94FD000E9418010E94180177
:101AA0001124F8941DBA109268001CBC10BE1FBA15
:101AB00010926E0010926F00109270001092C10090
:101AC0001092BC0010927A0014B817B81AB815B862
:101AD00018B81BB8099418954C4953206502525503
:101AE0004E209E045052494E990250525820A50251
:101AF000505242208404464F5220EB034E45585426
:101B0000D40253495A2079024E455720EF045050D1
:101B10000B205E0350500D20700350500A20270305
:101B200050500F203B03414F56201304454D49545C
:101B30006E04501A1D20B20250501D20BE02501CCF
:101B40001E20DD0250501E20D10350501C20C70320
:101B500050494620DF0350544F20ED0350500420DD
:101B6000F203454E4420F003414E442082034C537F
:101B700052208D034C534C209503504F52209D030F
:101B8000584F5220A803434F4D20B3034E454720E2
:101B9000BB03524E4420930444454C410004474F3C
:101BA000544F5E04474F53556304524554556704E0
:101BB0005448454EE7034B455920760441434F2096
:101BC000EE025341564551074C4F41448D07504555
:101BD000454BF702504F4B450D034F444220D3096C
:101BE00049444220CB0953444220E1094344422066
:101BF000F1094F504220010A53424220170A434242
:101C00004220270A494E42200F0A49424220370A01
:101C10004F444320D30949444320CB095344432034
:101C2000E10943444320F1094F504320010A534244
:101C30004320170A43424320270A494E43200F0AF4
:101C400049424320370A4F444420D30949444420A1
:101C5000CB0953444420E10943444420F1094F5047
:101C60004420010A53424420170A43424420270AD1
:101C7000494E44200F0A49424420370A44554D50EA
:101C800010054544554D60055644554DA505445332
:101C900052457C0B4453434F730B445344456A0BEA
:101CA000494347208B0A49434520AA0A494350200B
:101CB000C10A50574D385D0A50574520710A505798
:101CC0004F20870A44445320D40B424C44520D0DFC
:101CD00041444320860941445220B10953504D20CC
:101CE000040953504F2021095350432037095350C2
:101CF00057205309535052206109535053206D0906
:101D000054574920F00754575320B40854575020D3
:101D1000D008545741201808545757204C0854579E
:101D200052207C0854574220E60800000000F93C8D
:101D30003DFAF84174746F424153494320666F7213
:101D40002041546D65676131363820FAF856657266
:101D50003A20322E3131204275696C6420636F6401
:101D6000653A2032303132303330382E3033313230
:101D7000FAF93C2D0000F84F726967696E616C20BA
:101D8000636F646520284329323030322062792025
:101D9000526963686172642043617070656C73FAA4
:101DA000F8687474703A2F2F70726F6A6563747379
:101DB0002E63617070656C732E6F72672020707275
:101DC0006F6A656374734063617070656C732E6FC6
:101DD000726720FAF93C2DFAF854686520666F6C3A
:101DE0006C6F77696E672061726520656E68616EE1
:101DF00063656D656E74732062792053636F7474CC
:101E000020566974616C65FAF86B73765F70726A5C
:101E100040676D782E636F6D20FAF84D6567613805
:101E2000382F3136382F3332382F33325534207033
:101E30006F727420284329323031312C32303132E4
:101E400020FAF85457492F5350492F444453202621
:101E500020496E7075742043617074757265202816
:101E600043293230313120FAF84D656761333255FC
:101E7000342055534220262044465520426F6F742B
:101E80006C6F6164657220737570706F7274202856
:101E900043293230313220FAF93C2DFAF84D65678A
:101EA000613136382F33323820426F6F746C6F6176
:101EB000646572206261736564206F6E2073746B59
:101EC000353030626F6F742E63FAF8436F70797239
:101ED0006967687420286329323030332C204A61C6
:101EE000736F6E20502E204B796C65FAF93C2DFAF9
:101EF000F8416C6C2072696768747320616E6420AD
:101F000072656D6564696573206578707265737359
:101F10006C79207265736572766564FAF84E6F7439
:101F200020666F7220636F6D6D65726369616C20EE
:101F3000757365FAF93C3DFA0000F9352DFA000099
:101F40005661726961626C657320696E2052414D01
:101F50003AFA000045455020436F6E74656E747305
:101F60003AFA000050524F4752414D204D656D6F77
:101F7000727920436F6E74656E74733AFA000000D4
:101F80004E65787420617661696C61626C65206C65
:101F90006F636174696F6E3A20000000FB3A205055
:101FA000726F6772616D20746F6F206C617267650C
:101FB00020666F722045455021FA00005361766912
:101FC0006E6720746F204545502EFA000000FB45D7
:101FD00045502065726173656421FA0000004C6F02
:101FE0006164696E672066726F6D20454550FA0026
:101FF0000000427265616BFA0000467265653A2026
:1020000070616765733A00002063686172733A001B
:102010000000FA496E766F6B696E6720626F6F74AD
:102020006C6F6164657220617420307800004572C5
:10203000726F72200000FB303A20556E6B6E6F7726
:102040006E20636F6D6D616E64206F72206F7065BE
:102050007261746F722E0000FB313A20456E636F1F
:10206000756E746572656420612076616C7565209B
:1020700074686174206973206E6F74206265747770
:1020800065656E203020616E64203235352E00008B
:10209000FB323A2050726F6772616D206D656D6F13
:1020A00072792069732066756C6C2E000000FB331A
:1020B0003A20456E636F756E7465726564206120A9
:1020C0006368617261637465722074686174206909
:1020D00073206E6F742061207265636F676E697A1A
:1020E000656420747970652E0000FB343A696E7463
:1020F00065726E616C206572726F72202D20627540
:1021000066666572206C696D6974206578636565C3
:10211000646564000000FB353A20496E617070729E
:102120006F707269617465207661726961626C6555
:10213000206E616D6520656E636F756E7465726586
:10214000642E0000FB363A20446174612073746190
:10215000636B2070757368206572726F72202D201A
:10216000746F6F206D616E7920617267756D656E39
:102170007473206F6E206F6E65206C696E652E0023
:102180000000FB373A204461746120737461636B13
:1021900020706F70206572726F722EFAF9092046F6
:1021A000756E6374696F6E20747269656420746FF4
:1021B0002075736520612076616C75652074686197
:1021C0007420776173206E6F7420617661696C6131
:1021D000626C652E0000FB383A204D616368696EC1
:1021E0006520737461636B206572726F72FAF9090E
:1021F0002046756E6374696F6E7320616E642F6F15
:10220000722063616C6C73206E65737465642074F6
:102210006F6F20646565706C79206F7220746F6FCA
:1022200020636F6D706C65780000FB393A20474F72
:10223000544F206F7220474F53554220646573748A
:10224000696E6174696F6E206C696E652077617369
:10225000206E6F7420666F756E642E000000FB4167
:102260003A20537065636966696564206269742009
:10227000706F736974696F6E2072616E6765206F2D
:102280006620303A372065786365656465640000D0
:10229000FB423A204C696E65206E756D6265722056
:1022A000686173206D6F7265207468616E20746858
:1022B000726565206E756D6572616C730000FB431D
:1022C0003A205370656369666965642062697420A9
:1022D000706F736974696F6E2072616E6765206FCD
:1022E0006620303A31206578636565646564000076
:1022F000FB443A20537065636966696564206269CE
:102300007420706F736974696F6E2072616E676597
:10231000206F6620303A33206578636565646564B4
:102320000000FB453A20496E70757420436170745B
:10233000757265207265676973746572206F766562
:1023400072666C6F77000000FB463A204172697438
:10235000686D65746963206F766572666C6F77006F
:102360000000FB31303A2041726974686D65746910
:102370006320756E646572666C6F77000000FB31D8
:10238000313A20446976696465206279207A657201
:102390006F000000FB31323A2054574920627573B8
:1023A000206572726F72206F6363757265640000DE
:1023B000FB31333A2054574920696E746572666167
:1023C0006365206E6F7420656E61626C65640000E9
:1023D000FB31343A2054574920536C6176652072A2
:1023E00065706C6965642077697468204E414B00A4
:1023F0000000FB31353A204E6F20426F6F742D6C18
:0E2400006F6164657220666F756E6400000087
:103D000000000000000000000000000000000000B3
:103D100000000000000000000000000000000000A3
:103D20000000000000000000000000000000000093
:103D30000000000000000000000000000000000083
:103D40000000000000000000000000000000000073
:103D50000000000000000000000000000000000063
:103D60000000000000000000000000000000000053
:103D70000000000000000000000000000000000043
:103D8000FFFFFFFFFFFFFFFFFFFFFFFFFFFFFFFF43
:103D9000FFFFFFFFFFFFFFFFFFFFFFFFFFFFFFFF33
:103DA000FFFFFFFFFFFFFFFFFFFFFFFFFFFFFFFF23
:103DB000FFFFFFFFFFFFFFFFFFFFFFFFFFFFFFFF13
:103DC000FFFFFFFFFFFFFFFFFFFFFFFFFFFFFFFF03
:103DD000FFFFFFFFFFFFFFFFFFFFFFFFFFFFFFFFF3
:103DE000FFFFFFFFFFFFFFFFFFFFFFFFFFFFFFFFE3
:103DF000FFFFFFFFFFFFFFFFFFFFFFFFFFFFFFFFD3
:103E0000112484B714BE81FFF0D085E08093810037
:103E100082E08093C00088E18093C10086E08093B7
:103E2000C20080E18093C4008EE0C9D0259A86E06C
:103E300028E13EEF91E0309385002093840096BB0B
:103E4000B09BFECF1D9AA8958150A9F7CC24DD2404
:103E500088248394B5E0AB2EA1E19A2EF3E0BF2E27
:103E6000A2D0813461F49FD0082FAFD0023811F076
:103E7000013811F484E001C083E08DD089C0823420
:103E800011F484E103C0853419F485E0A6D080C024
:103E9000853579F488D0E82EFF2485D0082F10E0EE
:103EA000102F00270E291F29000F111F8ED0680127
:103EB0006FC0863521F484E090D080E0DECF843678
:103EC00009F040C070D06FD0082F6DD080E0C816C8
:103ED00088E3D80618F4F601B7BEE895C0E0D1E053
:103EE00062D089930C17E1F7F0E0CF16F8E3DF0614
:103EF00018F0F601B7BEE89568D007B600FCFDCF14
:103F0000A601A0E0B1E02C9130E011968C911197C0
:103F100090E0982F8827822B932B1296FA010C01A0
:103F200087BEE89511244E5F5F4FF1E0A038BF07D0
:103F300051F7F601A7BEE89507B600FCFDCF97BE86
:103F4000E89526C08437B1F42ED02DD0F82E2BD092
:103F50003CD0F601EF2C8F010F5F1F4F84911BD0D7
:103F6000EA94F801C1F70894C11CD11CFA94CF0C53
:103F7000D11C0EC0853739F428D08EE10CD084E9ED
:103F80000AD086E07ACF813511F488E018D01DD0B0
:103F900080E101D065CF982F8091C00085FFFCCFD4
:103FA0009093C60008958091C00087FFFCCF809158
:103FB000C00084FD01C0A8958091C6000895E0E688
:103FC000F0E098E1908380830895EDDF803219F06E
:103FD00088E0F5DFFFCF84E1DECF1F93182FE3DF0A
:103FE0001150E9F7F2DF1F91089580E0E8DFEE2736
:063FF000FF270994040400
:00000001FF
